:100000000C94AC080C94E4080C94E4080C94E408F8
:100010000C94E4080C94E4080C94E4080C94E408B0
:100020000C94E4080C94E4080C945B1D0C949D1C47
:100030000C942E200C94E4080C94E4080C94E4082E
:100040000C94E4080C94E4080C94E4080C94E40880
:100050000C947C230C94E11F0C94E4080C94E408A9
:100060000C94E4080C94E4080C94E4080C94E40860
:100070000C94E4080C94E4080C94E4080C94E40850
:100080000C94E4080C94E4080C94E4080C94E40840
:100090000C94E4080C94E4080C94E4080C94E40830
:1000A0000C94E4080C94E4080C94E408ED10F010AF
:1000B00023114C1153115E11611161116111AD12C7
:1000C000AD121C121F122412481269126C126F1208
:1000D00090124314451453144D1450145D14871496
:1000E000EB145F15F314BD14C114F714C414FA14FF
:1000F0000515CF145515D3140915D7140D1537153B
:10010000DB1411154115E11417152115C814FE143F
:10011000CB140115E6141C152D154D154F15B914EA
:10012000EF14681591159715821588159D15A3155F
:10013000A915E01506160B16101615161A161F1619
:10014000241629162E163316F316F316261726171D
:10015000A917C717CD18CD18CC174018511851182A
:10016000AD1AD41A851CD41A851C201B431B851C70
:10017000391C491C00DA1281FFD9F1DB20A4A62E1C
:10018000AF00A0C0D30000A1C8D30000AED580A8A6
:100190003F408D1420001E0F0500047F3F1F643276
:1001A00014643214783C1E1E140A0500000000007E
:1001B000000000000000000000000000000000003F
:1001C000000000000000000000000000000000002F
:1001D000000000000000000000000000000000001F
:1001E000000000000000000000000000000000000F
:1001F00000000000000000000000000000000000FF
:1002000000000000000000000000000000000000EE
:1002100000000000000000000000000000000000DE
:1002200000000000000000000000000000000000CE
:1002300000000000000000000000000000000000BE
:1002400000000000000000000000000000000000AE
:10025000000000000000000000000000000000009E
:10026000000000000000000000000000000000008E
:10027000000000000000000000000000000000007E
:10028000000000804080000000000000000000002E
:10029000000000000000000000000000008040801E
:1002A000000000000000000000000000000000004E
:1002B000000000000000000000000000000000003E
:1002C000000000000000000000000000000000002E
:1002D000000000000000000000000000000000001E
:1002E000000000000000000000000000000000000E
:1002F000000000000000000000000080000000007E
:10030000000001020402010101010101FF000000DF
:10031000000000000000FF010101010101020402D0
:10032000010000000000008000000000000000004C
:1003300000000000000000000000000000000000BD
:1003400000000000000000000000000000000000AD
:10035000000000000000000000000000000000009D
:10036000000000000000000000000000000000008D
:100370000000000000000000000205F80502000077
:100380000000000080C0C0E0E07078383F1C0E0E16
:100390000EFE0E0E1E1C3F387870E0E0C08000009C
:1003A00000000000000205F8050200000000000047
:1003B000000000000000000000000000000000003D
:1003C000000000000000000000000000000000002D
:1003D000000000000000000000000000000000001D
:1003E000000000000000000000000000000000000D
:1003F00000000000000000000040A013A2424242A2
:1004000042424242FFFFFF000000FCFEFEC0C0C0AF
:10041000C0FF0000003E3E3C3C000001FFFFFF42E9
:10042000424242424242A213A040000000008040EB
:10043000404080000000000000000000000080C07C
:100440004040C0800000C04040C08000000000006C
:100450000000000000000000C040C00000000000DC
:1004600080C04040C080000080C04040C08000008C
:100470004040404040C00000000000F90808080863
:10048000080808087FFFFFC080800F1F1F010101BF
:1004900001FF0000001E1E0E0E80C0C0FFFF7F087F
:1004A00008080808080808F900000000001F31408B
:1004B0004E40311F0000611608166100001F3160B8
:1004C0004040602000007F4444643B000000000086
:1004D000000000000000000040407F40400000009D
:1004E000206444446E3B0000206444446E3B0000A2
:1004F0000000007E0301000000081423140800001F
:1005000000000000000001010307070FFE1E1C1C75
:100510001CFF1C1C1C1EFE0F070303010100000032
:100520000000000000040A110A040000000000009E
:1005300000000000000000000000000000000000BB
:1005400000000000000000000000000000000000AB
:10055000000000000000000000000000000000009B
:10056000000000000000000000000000000000008B
:10057000000000000000000000000000000000007B
:100580000000102844281010101010101F00001038
:100590002847281000001F101010101010284428A1
:1005A00010000000000000000000002020202000BB
:1005B000534352200020202020004341502000209F
:1005C000202020004E554D2000556E646566696EF2
:1005D0006564004261636B6C6967687400524742EE
:1005E000004D49534300484F4D45004C61796572B9
:1005F0003A20000A000A20202020204D4F442048A5
:1006000055452053415420564152002C002C002CBB
:1006100000436F6E663A008081828384858687CB33
:10062000CBCBCBCBCBCBCBC0C1C2C3C4A0A1A2A3ED
:10063000A4A5A6A7CBCBCBCBCBCBCBCBE0E1E2E346
:10064000E488898A8B8A8B8C8DCBCBCBCBCBCBCBE5
:10065000CBCCCDCECFD0A8A9AAABAAABACADCBCBDF
:10066000CBCBCBCBCBCBECEDEEEFF0000000000022
:10067000000000000000000000000000000000007A
:10068000000000000000000000000000000000006A
:100690007E0F00D4FFFFFFC70000007800000000BD
:1006A000000000002A2B28000000000000000000CD
:1006B0000000000000000029000000002C1E342073
:1006C000212224342627252E362D3738271E1F2099
:1006D0002122232425263333362E37381F040506DE
:1006E0000708090A0B0C0D0E0F1011121314151622
:1006F0001718191A1B1C1D2F3130232D3504050620
:100700000708090A0B0C0D0E0F1011121314151601
:100710001718191A1B1C1D2F3130354C0501090201
:10072000A10185020901A100050919012908150087
:1007300025019508750181020501093009311581EE
:10074000257F95027508810609381581257F950159
:1007500075088106050C0A38021581257F950175FB
:10076000088106C0C005010980A101850319012A7D
:10077000B700150126B700950175108100C0050C62
:100780000901A101850419012AA002150126A00270
:10079000950175108100C00660FF0961A101096221
:1007A000150026FF009520750881020963150026B3
:1007B000FF00952075089102C005010906A10105F9
:1007C0000719E029E71500250195087501810295B3
:1007D00001750881010507190029FF150026FF0092
:1007E00095067508810005081901290515002501E0
:1007F000950575019102950175039101C009025B90
:1008000000030100A0FA090400000103010100092E
:10081000211101000122440007058103080001099C
:10082000040100020300000009211101000122223D
:1008300000070582032000010705030320000109CA
:100840000402000103000000092111010001227BC4
:1008500000070584032000011201000200000008C7
:1008600000CB37130100010200010A0331003300FD
:100870003300370000000A033000780043004200D4
:100880000000040309040000000000003E5B4F5B11
:100890003E003E6B4F6B3E001C3E7C3E1C00183CF5
:1008A0007E3C18001C577D571C001C5E7F5E1C00A0
:1008B00000183C180000FFE7C3E7FF0000182418E9
:1008C0000000FFE7DBE7FF0030483A060E0026296C
:1008D00079292600407F05050700407F05253F0058
:1008E0005A3CE73C5A007F3E1C1C0800081C1C3E7A
:1008F0007F0014227F2214005F5F005F5F00060903
:100900007F017F00006689956A006060606060001A
:1009100094A2FFA2940008047E04080010207E2008
:10092000100008082A1C0800081C2A0808001E10CD
:10093000101010000C1E0C1E0C0030383E38300019
:10094000060E3E0E060000000000000000005F00E2
:100950000000000700070000147F147F1400242A01
:100960007F2A120023130864620036495620500083
:10097000000807030000001C224100000041221C67
:1009800000002A1C7F1C2A0008083E08080000807E
:1009900070300000080808080800000060600000CF
:1009A0002010080402003E5149453E0000427F40AD
:1009B00000007249494946002141494D330018144D
:1009C000127F10002745454539003C4A494931000E
:1009D000412111090700364949493600464949294C
:1009E0001E00000014000000004034000000000859
:1009F000142241001414141414000041221408009D
:100A00000201590906003E415D594E007C12111247
:100A10007C007F49494936003E41414122007F41E7
:100A200041413E007F49494941007F0909090100D0
:100A30003E41415173007F0808087F0000417F411B
:100A400000002040413F01007F08142241007F4008
:100A5000404040007F021C027F007F0408107F009E
:100A60003E4141413E007F09090906003E415121B6
:100A70005E007F09192946002649494932000301D1
:100A80007F0103003F4040403F001F2040201F00E7
:100A90003F4038403F0063140814630003047804A7
:100AA00003006159494D4300007F41414100020468
:100AB00008102000004141417F00040201020400AF
:100AC0004040404040000003070800002054547894
:100AD00040007F28444438003844444428003844C7
:100AE00044287F0038545454180000087E0902003E
:100AF0001824241C78007F080404780000447D40FA
:100B000000002040403D00007F10284400000041CC
:100B10007F4000007C04780478007C08040478009E
:100B2000384444443800FC1824241800182424189D
:100B3000FC007C08040408004854545424000404B5
:100B40003F4424003C4040207C001C2040201C00EE
:100B50003C4030403C004428102844004C10101009
:100B60007C004464544C44000008364100000000FE
:100B70007700000000413608000002010204020074
:100B80003C2623263C0000E0FC1E06C6C6061EFCD2
:100B9000E000000060E080000080E06000000000F5
:100BA000E0F83C0E0606060E0C000000FEFE8686EF
:100BB00086868C787000000E0E0606FEFE00000091
:100BC0000000000C8E8686868686CEFE7C0000069F
:100BD0000606060606E6E63E3E00010101010101A9
:100BE000010106788000000000000000E01C020106
:100BF0000418000000020C00808071021CE000005C
:100C000000000000008078060101010101010101DE
:100C1000F0F8F8F8F8F80000FCFCFCFCFCFEFEFE26
:100C2000FFFFFFFFFFFFFF00E0E0E0E0F0F000006B
:100C300040F0FCFFFFFCF0C00000FFFFFFFFFF00E3
:100C400000000000000000073F7860636360783FA9
:100C5000070000006079190606197960000000009D
:100C6000071F3C7060606070300000007F7F616132
:100C70006161311E0E0000606060607F7F606060B7
:100C800060000030716161616161737F3E0000004E
:100C90000000007F7F010100000000000000000054
:100CA0000000000003BC8080808080808738408006
:100CB0000808080404020201000080403887808090
:100CC00080808080BC03000000007F7F7F7F7F7F6B
:100CD0007F7F7F7F7F7F00007F7F7F7F7F7F7F7F22
:100CE0007F7F7F7F7F7F7F0000000000C0F0FCFEE1
:100CF000FCF8F9F3F7FFFFFFFFFCF0C00000000075
:100D000000000000000070D070000705070202829A
:100D1000C2427EC0C0C0407E42C2820202070507B6
:100D20000070D07000000080402010C8C884040209
:100D3000020202C2C2C2C2C4C4C88890204080005D
:100D4000000000000000000000000000000001FDA5
:100D5000050404041F3040879F1F0181FFFF00002E
:100D60001E9E8640301F04040405FD01000F7080A4
:100D70000000000080E0F83E0F0300FFFF010101CA
:100D800001010000000080700F00FEFEFEFEFEFE6E
:100D9000FEFEFEFEFEFE0000FEFEFEFEFEFEFEFE6F
:100DA000FEFEFEFEFEFEFE00C0F0FCFFFFFFFFFFAA
:100DB000FF070303030307FFFFFFDF9F3F3C704074
:100DC000000000000000C05FD0909090FC0601F889
:100DD000FCFCC0C0FFFF00003C3C300106FC9090D2
:100DE00090D05FC000F00E01000000000103071E5C
:100DF0003CF0E0FFFF80808080C1C1FF3E00010E1B
:100E0000F0000000000000000000000000000705E6
:100E10000700705070202020213F01619F9F6101D9
:100E20003F212020207050700007050700000001BE
:100E30000204081013232040404040434340402018
:100E400020101008040201000000070707070F0F19
:100E50000F1F1F1F1F1F00003F3F3F3F3F7F7F7F30
:100E6000FFFF0080C0707C3F3F1F0F0F0707070385
:100E70000302000000000203030707070F0F1E3ED6
:100E80003C7C70C0800000000000000000000000FA
:100E90000001010203040506080A0C0F1114181CB6
:100EA0002024292E33393F464C535B626A71798185
:100EB0008A929AA2AAB2B9C1C8CFD5DCE1E7EBF019
:100EC000F4F7FAFCFDFEFFFEFDFCFAF7F4F0EBE7A9
:100ED000E1DCD5CFC8C1B9B2AAA29A928A81797150
:100EE0006A625B534C463F39332E2924201C181468
:100EF000110F0C0A0806050403020101000000009E
:100F000000000000000000AF00AEAC00AB00AE007F
:100F10004B004E0003524A004D00015201000100F7
:100F2000010001000100005201000100025223787B
:100F30002478217825782678015229782A78035256
:100F400005780678027800780178025204780378F0
:100F50000052FFAA7F55402223252628292A2C2D1E
:100F60002F3032333536383A3B3D3E4042434547D9
:100F7000494A4C4E5051535557595A5C5E60626411
:100F80006668696B6D6F71737577797B7D7F81831F
:100F90008587898A8C8E90929496989A9C9E9FA120
:100FA000A3A5A7A8AAACAEAFB1B3B4B6B8B9BBBC41
:100FB000BEBFC1C2C3C5C6C7C9CACBCCCDCED0D1B6
:100FC000D2D2D3D4D5D6D7D7D8D9D9DADADBDBDBAE
:100FD000DCDCDCDCDCDDDDDDDDDCDCDCDCDCDBDB4F
:100FE000DBDADAD9D9D8D7D7D6D5D4D3D2D2D1D0A3
:100FF000CECDCCCBCAC9C7C6C5C3C2C1BFBEBCBBA0
:10100000B9B8B6B4B3B1AFAEACAAA8A7A5A3A19F17
:101010009E9C9A98969492908E8C8A8987858381DB
:101020007F7D7B79777573716F6D6B6968666462BC
:10103000605E5C5A5957555351504E4C4A4947458A
:101040004342403E3D3B3A3836353332302F2D2C2B
:101050002A2928262523220001010101010101017D
:10106000010202020202020202020303030303035B
:101070000303040404040404040505050505060629
:1010800006060607070707070808080809090909E7
:101090000A0A0A0B0B0B0C0C0C0D0D0D0E0E0E0F8D
:1010A0000F0F10101111111212131314141515161D
:1010B000161717181819191A1A1B1B1C1D1D1E1E8E
:1010C0001F202021222223242425262627282929DF
:1010D0002A2B2C2D2D2E2F3031323233343536370A
:1010E00038393A3B3C3D3E3F404142434445464708
:1010F00048494A4C4D4E4F50515354555658595AE1
:101100005B5D5E5F616264656668696B6C6D6F7084
:1011100072737577787A7B7D7E8082838587888AF3
:101120008C8E8F91939596989A9C9EA0A2A3A5A72A
:10113000A9ABADAFB1B3B5B7BABCBEC0C2C4C6C926
:10114000CBCDCFD1D4D6D8DBDDDFE2E4E7E9EBEEDF
:10115000F0F3F5F8FAFDFF0011241FBECFEFDAE03F
:10116000DEBFCDBF04B603FE18C080910207909188
:101170000307A0910407B09105078730904BA74063
:10118000B04B59F410920207109203071092040713
:1011900010920507E0E0F8E3099511E0A0E0B1E066
:1011A000EEE1FEE602C005900D92A43CB107D9F72E
:1011B00027E0A4ECB1E001C01D92A230B207E1F734
:1011C0000E94E6080C940D370C940000AAE2B0E0EF
:1011D000ECEEF8E00C94193585B7806885BF85B7CB
:1011E000806885BF84B7877F84BF0FB6F894A895C1
:1011F00080916000886180936000109260000FBE53
:1012000090E080E80FB6F8948093610090936100BD
:101210000FBE81E08093180180E294E29093C501B3
:101220008093C4010E94E11C0E94001D8091E20095
:1012300084608093E200789480912E028823A1F04C
:101240001091E9001F709091EC00892F817090FD42
:1012500080E8182B1092E9008091E80083FD0E943D
:10126000C5191F701093E90082E084BD93E095BD1D
:101270009AEF97BD80936E000E94FA20811102C000
:101280000E94622288E0E5E5F6E0DF011D928A9582
:10129000E9F781E08093D50160E080E00E94AF2211
:1012A00061E080E00E94AF22EFE8F1E03197F1F7D2
:1012B00000C0000010E08091D501181790F460E0A4
:1012C000812F0E94A022082F61E0812F0E94A0227E
:1012D000E12FF0E0EC52FE4F880F082B00831F5FD8
:1012E000EACF48E251E0A1E0B0E020E030E0FA01CE
:1012F000E20FF31F80818F3FA1F0E82FE295EF709E
:10130000F0E061A18F708D0102C0000F111F8A955E
:10131000E2F7C801902F9095962391A392A1892B73
:1013200082A32F5F3F4F2330310509F74D5F5F4F99
:1013300011E041335107C9F683E0EEE1F2E0DF014D
:10134000082F1D920A95E9F7E6ECF1E0DF011D9206
:101350008A95E9F780E090E00E94C335853E9E4F74
:1013600021F40E94FA20811163C065EE7EEF80E0D7
:1013700090E00E94F73560E082E090E00E94D9356D
:1013800081E08093C90161E083E090E00E94D9355B
:1013900060E074E184E090E00E94F73560E086E070
:1013A00090E00E94D93560E087E090E00E94D93556
:1013B00040E050E0BA0188E090E00E94EB3560E048
:1013C00083E290E00E94D93560E08CE090E00E94DA
:1013D000D93560E08DE090E00E94D93519821A82FB
:1013E0001B821C821D821E821F82188648E050E0EC
:1013F00067E170E0CE0101960E94C93540E050E0FF
:10140000BA018FE190E00E94EB3580E00E94DB2082
:101410000E94622240E050E0BA018FE090E00E941A
:10142000EB3540E050E0BA0183E190E00E94EB35FB
:1014300082E090E00E94B5358093CF0184E090E097
:101440000E94C3359093CB018093CA010E94F72874
:10145000EFEFF6E701E0E150F0400040E1F700C0B7
:1014600000000E94F72880911E0280FF08C06FEFE5
:101470007FEF80E090E00E94F7350E94BD1F83E07F
:1014800090E00E94B5350E94072F259A2D9882E89A
:101490008093800089E1809381008FEF9FEF90938C
:1014A0008700809386000E94AD2A80914B0681FFC1
:1014B0000BC010924E0610924D0610924C06809171
:1014C0006F00816080936F000E9422209093D90169
:1014D0008093D80110921B0280E8809338020E940A
:1014E000EB336BE070E08BE891E00E942F238823C0
:1014F00089F180911B0265E070E081FD28C086E8DB
:1015000091E00E942F23882329F16DE070E084E7A9
:1015100091E00E942F238823E9F00E941620DC012D
:10152000CB01805A9541AF4FBF4F80934F069093A8
:101530005006A0935106B09352060E941A2381E0F0
:10154000809354068093530610921C0203C081E8D6
:1015500091E0D7CF0E94AD2A8091CC01811182C049
:1015600088E090E00E94BD354B015C0183E290E091
:101570000E94B535282F30E040E050E060E070E098
:1015800080E090E000E20E94BC36282939294A29EF
:101590005B292093F4063093F5064093F6065093AA
:1015A000F7066093F8067093F9068093FA06909315
:1015B000FB062C7F09F044C029E02093F40638E9AB
:1015C0003093F50638EE3093F6063FEF3093F7068A
:1015D00032E03093F80638E948EE5FEF62E00E94AF
:1015E000943188E090E00E94BD356B017C0183E27C
:1015F00090E00E94B535282F30E040E050E060E0F8
:1016000070E080E090E00E94BC36B22FA32FF42F50
:10161000E52F5B0197018601BC29A12BF22BE32B5F
:10162000B093F406A093F506F093F606E093F70660
:101630006093F806B092F9068093FA069093FB0641
:101640000E9480311092DD060E94841E8091F40673
:1016500080FF05C060E0869586950E94BA3181E0E2
:101660008093CC0184E091E090937C0680937B068C
:10167000DD24D3946624639444244394512CBE0106
:101680006F5F7F4F7B0180912E02853009F066C02D
:1016900010E402E180912E02853009F050C0809163
:1016A0002E02843009F43BC080E00E94272A109269
:1016B000DD068091CE0181110DC0D092CE018091C6
:1016C000F406982F91709093CD018E7F8093F4064D
:1016D0000E94D42A0E943C2310927F0688E190E069
:1016E0000FB6F894A895809360000FBE1093600029
:1016F00083B7817F846083BF83B7816083BF789421
:10170000889583B78E7F83BF0FB6F894A895809194
:101710006000886180936000109260000FBE0E949C
:10172000F72880911E028111ACC180911F028111A6
:10173000A8C180912002882309F4ACCFA2C10E94E5
:101740002D2F0E94AD2A0E94C6201092CE018091BA
:10175000CD0181110E94FF310E942F2E0E94F72897
:1017600000ED11E02EE1A22E22E0B22E23ED31E0B9
:10177000D501F80191918D9189272E173F0719F016
:101780008823C1F306C0811104C00E94D328C12C54
:1017900033C0C12CD5013D905D01F80170807324E8
:1017A00009F1912C88248394872D8821A1F099A296
:1017B000CAA20E9422209CA38BA36DA291E0832D3C
:1017C000882109F490E09EA349A15AA16BA17CA1B4
:1017D0008DA10E94F2329394880CF3E09F12E4CF23
:1017E000D8013C92C3940F5F1F4FB3E0CB12D2CF0E
:1017F0000E941620CC24C3948091DD06882309F42E
:10180000A6C08091DC06E091F406E695E695E81B1B
:10181000E093D806823059F4F0E0E955FE4FE491A8
:101820000E2F10E091E5A92E9DE2B92E6BC08630F7
:1018300059F4F0E0EC55FE4FE4910E2F10E081E4F6
:10184000A82E8DE2B82E5EC0893061F4E695F0E0F6
:10185000EF55FE4FE4910E2F10E0BDECAB2EBCE235
:10186000BB2E50C08F3061F4E695F0E0E256FE4F9B
:10187000E4910E2F10E0A2E7AA2EACE2BA2E42C0ED
:10188000853159F4F0E0E556FE4FE4910E2F10E05B
:10189000F6E2AF2EFCE2BF2E35C08831F9F083327C
:1018A00049F4E9E9F1E005911491E4E1AE2EEDE2AD
:1018B000BE2E28C08432C9F08532F1F48E2F63E049
:1018C0000E948036E92FF0E0EA56FE4FE4910E2F99
:1018D00010E07CEEA72E7AE2B72E14C008E210E0EA
:1018E0006DEAA62E6BE2B62E0DC004EF11E05EE7A6
:1018F000A52E5BE2B52E06C000ED17E047E7A42E4B
:1019000049E2B42E8091D906882361F01092D9065D
:101910000E9422209093D7068093D6061092DB0671
:101920001092DA060E942220E091D606F091D706A6
:101930008E1B9F0B8F3F9F4750F40E0F1F1F10935E
:10194000D7060093D60686ED96E0F50109958091BD
:10195000D601882351F01092D601809157068093CA
:1019600058068091550680935606B12C8091D5017A
:10197000B81608F040C061E08B2D0E94A022182FFD
:1019800060E08B2D0E94A022E12FEE0F8E2B0B2DFD
:1019900010E0D801AC52BE4FEC912E2F237030E0F6
:1019A000482F50E02417350721F1EE0FEE0FE82BFA
:1019B000EC93EF70F0E0EF5CFE4F0D521E4FA080F5
:1019C000D8018C91A80EAC92B3E0BA1514F460E083
:1019D00004C0EDEFAE1624F461E08B2D0E94C52209
:1019E0008A2DAA0C990B64E070E00E948C36D80115
:1019F0008C93B394BBCF90E080915806209157060A
:101A0000281709F465C0E82FF0E0E75AF94F208164
:101A100027FB222720F98F5F8370809358068091DF
:101A200056068F5F809356068091D7018823F9F080
:101A300090E0AC01559547955595479540FF08C0F6
:101A4000222319F00E94222E38C00E94152E39C080
:101A500003E0959587950A95E1F780FF08C022235A
:101A600019F00E94892A29C00E94662A2AC02223CE
:101A700021F089EA0E94483120C08AEA0E94483158
:101A800020C080912D02882309F404CE90E199BDF5
:101A900009BD09B400FEFDCF8091D8008F7D8093F1
:101AA000D8008091E00082608093E0008091E000A7
:101AB00081FDFCCF0E942D2FEDCD6AE070E089EA18
:101AC00003C06AE070E08AEA0E94303191E094CF6E
:101AD000992321F00E941620CC24C39480915406AF
:101AE000882309F427C28BE392E090934206809307
:101AF00041068091DA0181114EC08091D801909108
:101B0000D9010E940720883E934008F040C0809190
:101B10004106909142068B5392409C013C5F2130DC
:101B2000344028F020E034E0281B390B02C020E0CC
:101B300034E06091390270913A02DC01A55CBD4F3E
:101B4000AC01280F391F42175307E0F4FA01E81BD4
:101B5000F90BE555FE4FE491FC91EF1779F0EC930A
:101B6000FA0116E0F695E7951A95E1F7820102C0B1
:101B7000000F111FEA95E2F7602B712B4F5F5F4F4B
:101B80001196E1CF70933A0260933902C9C00E9466
:101B90001A23D092DA018BEE95E00E949919809178
:101BA000D7010E94B932813059F038F0823059F0B3
:101BB000833061F483ED95E00BC086EE95E008C0BC
:101BC00081EE95E005C08DED95E002C089EC95E0D1
:101BD0000E94A7190E94D320182F80FF03C084EC15
:101BE00095E002C08FEB95E00E94991911FF03C0A8
:101BF0008AEB95E002C085EB95E00E94991912FFEF
:101C000003C080EB95E002C08BEA95E00E94A71923
:101C10001091F40610FF7CC08091D7010E94B93268
:101C2000823009F075C016951695812F90E01C82C0
:101C30006AE070E00E940535805D8B836115710557
:101C400011F0605D01C060E26A8380E2898381E116
:101C500096E00E949919C7010E94AD198091F5067E
:101C600086958695869590E01C826AE070E00E94D9
:101C70000535805D8B836115710511F0605D01C0D4
:101C800060E26A8380E289838FE096E00E9499197E
:101C9000C7010E94AD198091F606869586958695B6
:101CA00090E01C826AE070E00E940535805D8B83C5
:101CB0006115710511F0605D01C060E26A8380E228
:101CC00089838DE096E00E949919C7010E94AD19A1
:101CD0008091F70686958695869590E01C826AE04D
:101CE00070E00E940535805D8B836115710511F0F0
:101CF000605D01C060E26A8380E289838BE096E0E8
:101D00000E949919C7010E94AD1985EF95E002C0A4
:101D100083EF95E00E94A71987E196E00E94991948
:101D20008091390290913A02892B31F480915306C7
:101D3000882309F4FFC0E7C0809154068823B1F3DB
:101D400080911C028111F2CF0E945623209139020A
:101D500030913A022115310549F380E0082F10E057
:101D60005201082E02C0AA0CBB1C0A94E2F7A5017E
:101D700042235323452B11F48F5FF0CF90911B0228
:101D8000980166E0220F331F6A95E1F790FF13C0B8
:101D900056E0369527955A95E1F7220F220F220F2C
:101DA0002093100110921301295F2093110187E005
:101DB0008093140112C0220F232F221F330B319561
:101DC0008295880F880F80748093100120931301EF
:101DD000815C809311012093140124E630E047E0F8
:101DE00050E06EE071E088E70E942034892B09F012
:101DF0009DCF80911B0280FF66C080E4EBEDF1E097
:101E0000DF011D928A95E9F7180196E0220C331C38
:101E10009A95E1F7E9E4F1E0FAA7E9A741E451E096
:101E2000A9A5BAA58D91BAA7A9A7FA019191AF0169
:101E30009101290F311D8901055C1D4F18A70FA3C2
:101E400090E085529E4FFC0107E09F01281B390B53
:101E5000842C01C0880C2A95EAF76FA178A5912CF3
:101E6000DB011D91BD011821202F29192770722E29
:101E7000022E000C330BB12F01C0BB0F7A94EAF78E
:101E80007B2E3195219531092770332701C0169596
:101E90002A95EAF7712A1081712A7082939418E0CA
:101EA0009112DECF015031960F3F79F669A57AA5E0
:101EB0006155714009F0B4CF04E610E020E430E051
:101EC0004BED51E00CC0A80186E0440F551F8A95E8
:101ED000E1F7455C5D4F04E610E020E430E060E4AB
:101EE00088E70E94B734892B09F020CFA094B094E2
:101EF0008091390290913A02A822B922B0923A0216
:101F0000A092390213CF0E94162000914F06109123
:101F100050062091510630915206DC01CB01801B06
:101F2000910BA20BB30B8F3F9F4FAF4FBF4710F4E6
:101F30000E943C23C1100E94562386E0E0E7F6E0B1
:101F4000D70101900D928A95E1F7A090710600915A
:101F5000720610917306C0907406B09075061092C8
:101F60007206109273061092740610927506011193
:101F700003C0112309F44BC080916E0690916F0647
:101F80000E9407209C0190916906992309F4F7C2E9
:101F900025313105E0F19F3F19F09F5F909369066D
:101FA000002361F00E94C821101614F491E001C0D2
:101FB0009FEF899F802D112480937206112361F079
:101FC0000E94C821111614F09FEF01C091E0899F73
:101FD000802D112480937306809172068823B9F0B6
:101FE00090907306992099F00E94E821882319F0B7
:101FF0008093720602C0D0927206892D0E94E82159
:10200000882319F08093730602C0D0927306C11022
:1020100003C0BB2009F44BC080916C0690916D0603
:102020000E9407209C0190916A06992309F4ACC292
:1020300021353105E0F19F3F19F09F5F90936A06CB
:10204000CC2061F00E94A6211C1414F491E001C080
:102050009FEF899F802D112480937406BB2061F02F
:102060000E94A6211B1414F09FEF01C091E0899FEC
:10207000802D112480937506809174068823B9F011
:1020800090907506992099F00E94E821882319F014
:102090008093740602C0D0927406892D0E94E821B4
:1020A000882319F08093750602C0D092750680913E
:1020B00071068A111AC080917206882311F080136C
:1020C00014C080917306882311F018130EC08091FC
:1020D0007506882311F08B1108C09091740699231E
:1020E00031F081E09C1104C002C081E001C080E0B9
:1020F00080FD15C08091720681110FC0809173061A
:1021000081110BC080917406811107C081E090910C
:102110007506911103C080E001C081E080FD0E943E
:102120007C21AA820B831C83CD82BE8286E0F701CC
:10213000A0E7B6E001900D928A95E1F70E94C620D3
:1021400090911D02891721F080931D020E94162094
:1021500080912E02843009F096CA83E08093E900D2
:102160008091E80082FF8FCA8091E80085FF1FC040
:102170000E94411E811119C000E210E0570108C001
:102180008091F100D5018D935D010150110969F035
:102190008091E80085FDF4CF8091E8008B778093F3
:1021A000E8000E94411E882399F391E001C090E06D
:1021B0008091E8008B778093E800992309F463CA43
:1021C0002981822F90E0FC013197E331F10508F07D
:1021D000C4C1EA5AFF4F0C94A0361A828CE032C177
:1021E0008A81823009F4C2C150F4813009F0B5C14E
:1021F0000E9416209B838C837D836E83B0C18330C5
:1022000041F0843009F0A9C11B821C821D821E820C
:10221000A6C14B81DE01149680E090E0242F30E0CF
:10222000B901680F791F6330710508F098C1E42F78
:10223000E80FF0E0E25EFD4F50815D9301968C3136
:10224000910571F78CC18A81823019F0853051F087
:1022500084C16B817C818D819E810E94A6360E9403
:10226000D6207DC180914B0680FF03C00E94412A89
:1022700002C00E944E2A8091F40680FF0AC080911D
:10228000F4068E7F8093F4061092DD060E94D42A15
:1022900066C10E94FF3163C14C816B818A810E94BB
:1022A00072229D836AC12D813E81322723273227E6
:1022B0004C816B818A810E94062251C10E942D228D
:1022C0004EC18A818130E1F52830F1F0293099F151
:1022D0008B81813019F0823071F041C18C81B7E07F
:1022E0008B9FC00111246FEF70E00E940535862F8F
:1022F0000E94272A34C18C81811103C00E94FC29CD
:102300002EC10E94122A2BC18B81813041F0823074
:1023100009F025C180914B068695817078C0809127
:102320004B06869586958695EFEF8E9FC00111240A
:1023300067E070E05DC080914B060E94F6290FC1F6
:10234000823009F00AC12830B9F1293009F461C09E
:102350008B818230F9F098F4813009F000C18C81D2
:10236000FFEF8F9FC00111246FEF70E00E940535D1
:10237000462F20E06091F6068091F5061AC0833062
:10238000A1F0843009F0EBC020E04091F7066D81A8
:102390008C810FC08C81882309F471CF0E94FF319A
:1023A00060E08C810E94BA31DAC08C818093F8069B
:1023B000D6C00E94652DD3C08B818230E9F060F4D5
:1023C000813009F0CCC08091F7060FEF809FC001EB
:1023D00011246FEF70E00CC08330B9F0843009F045
:1023E000BEC08091F5068C838091F6068D83B7C0C0
:1023F0000E9405356C83B3C08091F40680FF03C052
:102400008695869504C080E002C08091F8068C8392
:10241000A6C02091F4063091F5064091F606509141
:10242000F7066091F8067091F9068091FA0690918E
:10243000FB060E94943193C010E11A8390C083E0A0
:102440008A8380E98B838BC00A811B811027012737
:102450001027AC80B12C4701C80180599F4F9401CF
:102460002E193F092A153B0508F079C0003923E0F1
:10247000120730F40E94B535D40114968C9302C033
:10248000F40114820F5F1F4FFFEF8F1A9F0AE4CFF2
:102490000A811B81102701271027AC80B12C47012E
:1024A000C80180599F4F94012E193F092A153B05F9
:1024B00008F055C0003923E0120728F4D40114961F
:1024C0006C910E94D9350F5F1F4FBFEF8B1A9B0A8B
:1024D000E7CF0E94F62143C084E08A8340C00A818E
:1024E0001B81102701271027AC80B12C4701C801A0
:1024F000889694012E193F092A153B0580F508346A
:10250000110528F40E94B535F401848303C0D40179
:1025100014961C920F5F1F4FBFEF8B1A9B0AE7CFD9
:102520000A811B81102701271027AC80B12C47019D
:10253000C801889694012E193F092A153B0578F4A5
:102540000834110520F4F40164810E94D9350F5F2D
:102550001F4FFFEF8F1A9F0AEBCF8FEF898340E267
:1025600050E0B70182E00E945D1F8DC887E290E0D5
:102570000E94B5351B821C821D828E83F0CF2B30CA
:10258000310508F00ACD43CD2B30310508F055CD8B
:102590008ECDA8E0B0E0EFECF2E10C941935FC012F
:1025A0008481882309F44AC67F0121E0408151815A
:1025B0006281738195810E94CD328C01F7019581F2
:1025C000992309F4AEC1980137572038310508F036
:1025D00050C1003108F0D6C28FEF93E00E94B535AC
:1025E0008111D0C230E7A32EB12C002379F0A114C1
:1025F000F4E0BF0609F4C6C2C5010E94B5358111D9
:1026000001C001502FEFA21AB20AEFCFCE010196FE
:102610002C0188E0F20111928A95E9F72AE0322E26
:1026200085010F5F1F4FC5010E94B53589831A824E
:10263000882309F4A7C2813009F041C06501F2E0A6
:10264000CF0ED11CC8010E94B5358A83882309F4B6
:1026500099C29FEF980F933060F423E0A20EB11C53
:10266000C6010E94B5358B83882309F48BC21C8276
:1026700029C0843031F54E0133E0830E911C02E015
:1026800010E056018FEFA81AB80AC6010E94B535AE
:10269000F40181934F01882309F474C28C3741F40B
:1026A000E2E0F0E0EC0FFD1FE00FF11F10820AC026
:1026B0000F5F1F4F65010730110519F763C25801FD
:1026C00001C056018201F8012081222309F4A8CF1C
:1026D000213009F050C08181813049F46801F2E075
:1026E000CF0ED11CF80182810E9448310AC082308D
:1026F00051F46801F2E0CF0ED11CF80182810E94F2
:102700009730860133C0833049F46801F2E0CF0E80
:10271000D11CF80182810E943D30F3CF843019F042
:102720000F5F1F4F23C0F80122810E5F1F4F80E013
:1027300090E030E0205331092A30310568F4389EAA
:10274000A001399E500D1124C901840F951F0F5F00
:102750001F4FF8012081EDCF009741F0EFE9FFE036
:102760003197F1F700C000000197F6CF8FE39CE9A5
:102770000197F1F779C0E22FF0E0E456F94F249089
:10278000822F86958695869590E0FC01E457F94F57
:1027900064902770712C022E02C0759467940A947D
:1027A000E2F7E1E06E227724FC01E458F94F8490CF
:1027B000912C022E02C0959487940A94E2F7F1E0DE
:1027C0008F229924FC01E459F94FC490D12C02C006
:1027D000D594C7942A95E2F721E0C222DD24611442
:1027E000710449F081EE0E9497308FE39CE90197D4
:1027F000F1F700C000008114910449F086EE0E94B8
:102800009730EFE3FCE93197F1F700C000006AE090
:1028100070E0822D0E9430318FE39CE90197F1F73F
:1028200000C000008114910449F086EE0E943D3002
:10283000EFE3FCE93197F1F700C000006114710487
:1028400049F081EE0E943D308FE39CE90197F1F75A
:1028500000C00000C114D10449F08CE20E9448314C
:10286000EFE3FCE93197F1F700C000000F5F1F4F65
:102870002ACFF801F857E730F10508F052C0E759C0
:10288000FF4F0C94A03687E001C080E00E94272A09
:1028900080914B060E94F62975C10E94662A72C17A
:1028A0000E94892A6FC180914B0680FF03C00E945D
:1028B000412A68C10E944E2A65C190914B06892F1A
:1028C0008695869586958F5F8F719770883038F4DE
:1028D000880F880F880F892B80934B0602C0909336
:1028E0004B0680914B06887F91E009F490E080913F
:1028F0004B0690FB80F980934B060E94F62980914D
:102900004B068695869586950E94F5233BC180915E
:102910004B0681FF03C00E94FC2934C10E94122A89
:1029200031C1F801E851FC47E730F10508F4E6C091
:10293000992309F45CC41092780698013057233229
:10294000310508F00CC184E090E00E94C3359093FB
:10295000CB018093CA01F801E150F047E232F10562
:1029600020F4E059FF4F0C94A0368091CA01816099
:10297000ACC08091CB018860B4C08091CA018260F4
:10298000A4C08091CA0120C08091CA0188609DC006
:102990008091CB011EC08091CB018260A2C080914A
:1029A000CA01806192C08091CA0180628EC080910C
:1029B000CA0180648AC00E942D2F8091CA0180685C
:1029C00084C08091CA01886084607FC08091CB01FF
:1029D0008260816086C08091CA018E7F76C08091BE
:1029E000CB01877F7EC08091CA018D7F6EC08091B0
:1029F000CA0120C08091CA01877F67C08091CB0146
:102A00001EC08091CB018D7F6CC08091CA018F7EEA
:102A10005CC08091CA018F7D58C08091CA018F7BB4
:102A200054C00E942D2F8091CA018F774EC0809193
:102A3000CA01877F8B7F49C08091CB018D7F8E7FBC
:102A400050C08091CA0182FB222720F991E0922791
:102A500090FB82F990FB83F938C08091CB01982FCD
:102A6000909591708E7F892B90FB81F93AC080916F
:102A7000CA0186FB222720F991E0922790FB86F974
:102A800024C00E942D2F8091CA0187FB222720F9A4
:102A900091E0922790FB87F918C061E001C060E0E7
:102AA0008EE090E00E94D9351EC08091CA0184FB5F
:102AB000222720F991E0922790FB84F906C08091AB
:102AC000CA01982F909590FB80F98093CA010BC0A2
:102AD0008091CB0183FB222720F991E0922790FB84
:102AE00083F98093CB016091CA017091CB0184E09E
:102AF00090E00E94F7350E942D2F44C0EE56FF4F04
:102B00000C94A03606E221EE41EE6AE17CE705C0B6
:102B100007E225EE45EE6BE17CE7C7010E94132139
:102B200031C006E221EE40EE68E17CE7F6CF07E235
:102B300025EE44EE69E17CE7F0CF06E221EE42EEBD
:102B40006CE17CE7EACF07E225EE46EE6DE17CE73B
:102B5000E4CF08E221E045EE6EE17CE7DECF809134
:102B6000D0060631FCE71F07F9F48A7A91E009F4F0
:102B700090E090932102811138C389E20E94632082
:102B80000E945F268091C506877009F457C3F7013C
:102B90008581882309F452C38091CB0182FF4EC303
:102BA00082E00E9499264AC38272F801E052F847F7
:102BB000EB30F10508F05CC0E756FF4F0C94A036EF
:102BC0008091F40680FF19C0282F2E7F2093F406F1
:102BD0003091F5064091F6065091F7066091F8069F
:102BE0007091F9068091FA069091FB060E9494314B
:102BF0001092DD060E94D42AC5CF81608093F4062E
:102C000061E0869586950E94BA31BCCF882329F071
:102C10000E940A32B7CF8823D9F30E941532B2CF6F
:102C2000882329F00E946C31ADCF8823D9F30E940C
:102C30007631A8CF882329F00E945231A3CF882370
:102C4000D9F30E945F319ECF882329F00E94152E70
:102C500099CF8823D9F30E94222E94CF882329F07C
:102C60000E94E12D8FCF8823D9F30E94FB2D8ACFBC
:102C70000737FCE71F0711F481E0D5C208372CE7BE
:102C8000120709F4CFC29801205E32452032310587
:102C9000A8F4911115C00F7181E090E09C0102C071
:102CA000220F331F0A95E2F78901622F83E090E03B
:102CB0000E94D935802F0E94072F64CF9923E9F114
:102CC00003303CE7130729F148F401159CE7190785
:102CD00091F00130ECE71E0711F12FC00B35FCE736
:102CE0001F0741F10C352CE71207E1F00A351C47AC
:102CF00021F581E020C00E942D2F8FEF94E3ECE0BE
:102D000081509040E040E1F700C000000E94BD1FEC
:102D100039CF6FEF7FEF80E090E00E94F7350E949F
:102D2000823330CF8091CB0182FB882780F991E0FC
:102D3000892701C080E00E94B026F70185810081CB
:102D40001181882349F0C8010E94462ED82E682F91
:102D5000C8010E94B62E04C0C8010E94822ED82E3F
:102D6000B8018D2D0E942D250E943B25D82E192FAC
:102D7000A82EF7010581C680C2949FE0C9228091E8
:102D8000C506877001F10023F1F0812F807F803428
:102D900069F080E28D0D8830B0F0812F807E803226
:102DA00029F4F1E0FD1578F4CC2069F08091CB0195
:102DB00082FF09C082E00E9499268091C506877033
:102DC000BB24B3948111B12C912E92948FE0982260
:102DD000892D90E08C30910508F0DFC1FC01EC55A5
:102DE000FF4F0C94A036812F807F1F70882311F035
:102DF0001295107F0023B9F0112309F4B7C180E2C6
:102E00008D0D883010F0A11006C09091D006192BBE
:102E10001093D00605C09091C706192B1093C706D2
:102E20000E945F26A3C18D2D0E943D30112309F41D
:102E3000B4C180E28D0D883088F1AA2079F1109517
:102E40009091C70619231093C7062BC0812F807F4E
:102E50001F70803211F01295107F8D2DAA2029F05D
:102E600021E0A21609F44CC057C08091CB0182FD2D
:102E70001BC0002369F0112339F09091D006192B63
:102E80001093D0060E945F2680E00E94973085C193
:102E900080E00E943D30112309F47FC1812F0E9400
:102EA00058260E945F2679C1002381F0CC20C1F111
:102EB00031E0C31272C19091C606812F8923181781
:102EC00009F46BC1192B1093C60667C1C11065C107
:102ED000812F0E94542F8091C606912F982329F0AC
:102EE000912F909589238093C60620912202812FED
:102EF000822309F452C110952123209322024DC14F
:102F0000002329F085E08C1508F447C109C094E03E
:102F10009C1508F442C119C0002331F0C11026C12C
:102F2000812F0E945B2F39C1CC2079F0893341F485
:102F3000EFEFF7EE23E0E150F0402040E1F728C149
:102F40008FE39CE90197F1F723C1812F0E94542F51
:102F500024C1812F86958695837019F0813061F0A8
:102F60001CC1002321F08D2D912F937002C080E0B1
:102F700090E00E94A12017C1002321F08D2D912FF8
:102F8000937002C080E090E00E947C200CC1602F12
:102F90008D2D0E94652F07C1812F8370A9F5011126
:102FA00000C14D2D429546954770440F440F8D2D1D
:102FB0008F7090E09C01042E01C0220F0A94EAF762
:102FC000D4FE08C08FE090E001C0880F4A95EAF770
:102FD000809501C080E0169516951370123069F047
:102FE00088F49091C901113019F0822B892302C015
:102FF000922B892B0E94072FD4C0822B9091C9015C
:103000008927F8CF822BF6CF002319F0812F81700A
:1030100001C08695882309F4C4C04D2D429546957C
:103020004770440F440F8D2D8F7090E09C01042E4B
:1030300001C0220F0A94EAF7D4FE08C08FE090E0A6
:1030400001C0880F4A95EAF7809501C080E0169587
:1030500016951370123059F078F49091D701113011
:1030600019F0822B892309C0922B892B06C0822B51
:103070009091D701892701C0822B0E94EB2E91C02D
:103080001F70002339F0812F0E94FB2E8D2D0E948E
:103090005B2F87C08D2D0E94542F812F0E94EE2E12
:1030A00080C08D2D92EFA91681F19A1538F0E0EFCE
:1030B000AE1659F0F1EFAF1619F154C023EFA21676
:1030C00059F134EFA316C1F04DC0002381F084E024
:1030D0008C1508F462C01F7181E090E0012E01C0E0
:1030E000880F0A94EAF79091D701892720C095E0CC
:1030F0009C1508F452C0EFCF8091CB0182FD1AC01D
:10310000002329F0812F8F7120C00023D9F3812F54
:103110008F710E94EE2E41C0002341F01F7181E0AB
:10312000012E01C0880F0A94EAF701C080E00E94D6
:10313000EB2E33C0002361F0812F8F71E8E08E9F6A
:103140009001112423602093C5060E94FB2E25C008
:1031500081E00E949926F1E0FC15F8F482E00E94DB
:1031600099261BC0002321F0CC2061F28D2D8DCE3D
:10317000CC2069F2893341F42FEF37EE83E0215000
:1031800030408040E1F704C0EFE3FCE93197F1F70C
:1031900000C000008D2D0E943D3088EF890D8430E5
:1031A00010F40E94C620BB20A9F08091C50680FDC6
:1031B00011C0F70115828695869586950E94FB2E93
:1031C000C7010E94C9128091C5068695869586958D
:1031D0000E94EE2E20E0F7014081518162817381CF
:1031E000848195810E94CD3229C085E3C7CC063108
:1031F0008CE7180751F480912102811104C089E203
:103200000E945720BDCC85E3FBCF07372CE7120780
:1032100011F481E00BC008373CE7130709F033CD08
:1032200082E004C082E00E94FB2E02C00E94EE2ECB
:1032300043E062E081E00E94B128A4CC2896E2E15C
:103240000C943535CF93DF93682F8A3011F481E0E9
:1032500003C08D3021F480E00E94EA2267C0809193
:1032600041069091420626E0FC01ABE3B6E00190F6
:103270000D922A95E1F726E0629FB00111246A576A
:10328000774F46E050E00E94AC35C0914106D091A6
:10329000420646E050E0BE018BE396E00E94003714
:1032A000892B49F19E012B533240A90186E05695A6
:1032B00047958A95E1F781E090E0BC0102C0660F76
:1032C000771F4A95E2F74091390250913A02462B16
:1032D000572B2B5F3F4F66E0369527956A95E1F7B0
:1032E00002C0880F991F2A95E2F7842B952B9093A3
:1032F0003A02809339029E012553324040913802B0
:10330000642F70E0C9010E940535481B463010F457
:10331000240F311D211584E0380710F020E030E043
:10332000255C3D4F3093420620934106DF91CF91BB
:103330000895CF93DF93EC01FE018491882321F05F
:103340000E9422192196F8CFDF91CF9108950E9413
:10335000991981E00E94EA2208950F931F93CF9359
:10336000DF93EC01FC0101900020E9F78F0101508F
:103370001109C017D10720F489910E942219F9CFB1
:10338000DF91CF911F910F910895AAE2B0E0EBEC8D
:10339000F9E10C942835E0E3F2E088E392E0209133
:1033A000F10021938E179F07D1F78091310283306E
:1033B00009F463C030F4813071F0823009F4A2C0A6
:1033C000B9C08A3009F48EC08B3009F46EC08930E0
:1033D00009F0B0C020C080913002813A09F0AAC043
:1033E0008091E800877F8093E8008091340290917B
:1033F0003502892B21F468E084E292E003C060E0AA
:1034000080E090E070E00E94FF1E8091E8008B77E2
:103410008093E8008FC080913002813209F08AC029
:103420008091340290913502009719F0029709F0CB
:1034300081C08091E800877F8093E8008091E80058
:1034400082FD05C080912E028111F8CF73C02091BA
:10345000F3008091F20090E0922B029731F480917A
:10346000F100813011F0863021F48091F1008093D9
:1034700016018091E8008B7759C080913002813A23
:1034800009F058C08091340290913502892B09F0DF
:1034900051C08091E800877F8093E8008091E80028
:1034A00080FFFCCF809117013CC0809130028132B7
:1034B00009F040C08091340290913502892BD1F5FA
:1034C0008091E800877F8093E8000E94AB1E81E036
:1034D00090913202911101C080E0809317010E9407
:1034E0002D2F28C080913002813221F58091E80093
:1034F000877F8093E8000E94AB1E80913302809307
:10350000150118C080913002813AA1F48091E80041
:10351000877F8093E8008091E80080FFFCCF809156
:1035200015018093F1008091E8008E778093E80088
:103530000E94AB1E8091E80083FFE7C180913002BA
:1035400090913102492F50E04A30510508F0DDC119
:10355000FA01E055FF4F0C94A036803821F08238F4
:1035600009F0D3C108C080912C0290912D029923BB
:1035700089F082600FC0809134028F70873008F02C
:10358000C4C18093E9008091EB0085FB882780F916
:103590001092E9009091E800977F9093E800809363
:1035A000F1001092F10071C1282F2D7F09F0ADC1FB
:1035B000882319F0823061F0A8C1809132028130F5
:1035C00009F0A3C1933009F080E080932D022EC052
:1035D0008091320281112AC0809134028F702FEFC6
:1035E000280F263008F091C18093E9002091EB006C
:1035F00020FF1CC0933021F48091EB00806214C046
:103600009091EB0090619093EB0021E030E0A901F4
:1036100002C0440F551F8A95E2F74093EA001092CA
:10362000EA008091EB0088608093EB001092E90043
:103630008091E800877F8093E8000E94AB1E65C1FF
:10364000811163C1109132021F778091E30080786D
:10365000812B8093E3008091E800877F8093E800CE
:103660000E94AB1E8091E80080FFFCCF8091E300B8
:1036700080688093E300111102C082E001C083E002
:1036800080932E0242C18058823008F03EC12091C2
:103690003202309133022C3D53E0350779F583E057
:1036A0008A838AE289834FB7F894DE01139620E07B
:1036B0003EE051E2E32FF0E050935700E49120FF09
:1036C00003C0E295EF703F5FEF708E2F90E0EA301D
:1036D00010F0C79601C0C0968D939D932F5F243143
:1036E00049F74FBF8091E800877F8093E8006AE246
:1036F00070E0CE0101960E94FF1EB5C08091340299
:1037000090913502432F552743305105A9F068F4B5
:103710004130510509F408C14230510509F0F5C0A6
:103720008BE590E0EDEFF7E04BC04132510529F118
:103730004232510589F1E9C0C901992781309105CB
:10374000A1F058F0029709F0E0C0EAE6F8E0E49151
:103750008E2F90E0EAE6F8E030C0E2E8F8E0E4918D
:103760008E2F90E0E2E8F8E028C0E6E7F8E0E49188
:103770008E2F90E0E6E7F8E020C08330910508F056
:10378000C4C0880F991FFC01E65AFE4F0190F081DA
:10379000E02D89E090E014C08330910508F0B5C0B9
:1037A000FC01EE0FFF1FEC5AFE4F0190F081E02D5F
:1037B000DC01AF5ABE4F8C9190E0009709F4A5C090
:1037C0002091E800277F2093E80020913602309175
:1037D00037028217930708F49C0140E02115310558
:1037E00089F180912E02882309F43DC08530D9F1FA
:1037F0008091E80083FD37C08091E80082FD2FC0F2
:103800008091E80080FFEACF4091F3008091F200C0
:1038100090E0942B2115310559F08830910540F442
:1038200044914093F1003196215031090196F2CF35
:1038300041E0089709F040E08091E8008E7780939E
:10384000E800CCCF4111CDCF0AC080912E02882351
:1038500051F0853041F08091E80083FD04C08091F3
:10386000E80082FFF2CF8091E8008B778093E80038
:103870004CC0803809F049C08091E800877F809370
:10388000E80080912F028093F1008091E8008E770C
:10389000D2CE81113AC080913202909133029927A1
:1038A00002979CF58091E800877F8093E800109153
:1038B000320210932F020E94AB1E111106C080919C
:1038C000E30087FD02C081E001C084E080932E0206
:1038D00042E061EC81E00E94CA1E42E261EC84E0B9
:1038E0000E94CA1E42E261EC82E00E94CA1E42E2CD
:1038F00060EC83E00E94CA1E80912E02843011F099
:1039000081E001C082E0809318018091E80083FF8C
:1039100010C08091E800877F8093E8008091EB00E1
:1039200080628093EB0005C082E190E0E8E5F8E07A
:1039300047CFAA96E3E00C9444351F920F920FB63E
:103940000F9211242F933F934F935F936F937F9325
:103950008F939F93AF93BF93CF93DF93EF93FF9397
:10396000C091E900CF708091EC00D82FD17080FD1C
:10397000D0E81092E9008091F000877F8093F000FA
:1039800078940E94C5191092E9008091F000886037
:103990008093F000CD2BCF70C093E900FF91EF91A1
:1039A000DF91CF91BF91AF919F918F917F916F9157
:1039B0005F914F913F912F910F900FBE0F901F90ED
:1039C0001895E8EDF0E080818E7F80831092E20010
:1039D0001092DA001092E100A0EEB0E08C918160CC
:1039E0008C9380818F77808319BCA7EDB0E08C9198
:1039F0008E7F8C9380818F7E808310922302089526
:103A0000A0E0B0E0E6E0FDE10C942335C8EDD0E0A5
:103A100088818F7E8883E7EDF0E0808181608083FC
:103A200084E082BF81E08093230288818E7F888337
:103A300002EE10E0F80110821092DA0081EEC82E3A
:103A4000D12CF601108288818F77888388818068E5
:103A5000888388818F7D888319BC10922E021092F2
:103A60002F0210922D0210922C0290EEE92EF12CD2
:103A7000F70180818B7F808388818160888342E029
:103A800060E080E00E94CA1EF60180818E7F808304
:103A9000F801808181608083808188608083F70164
:103AA00080818E7F8083888180618883CDB7DEB7F7
:103AB000E8E00C943F351F920F920FB60F9211243D
:103AC0002F933F934F935F936F937F938F939F9326
:103AD000AF93BF93EF93FF938091E10082FF09C002
:103AE0008091E20082FF05C08091E1008B7F80938E
:103AF000E1008091DA0080FF2AC08091D80080FF29
:103B000026C08091DA008E7F8093DA008091D90000
:103B100080FF18C080E189BD82E189BD09B400FE43
:103B2000FDCF81E080932E028091230281110FC08E
:103B30000E94E11C0E94001D8091E200846080933D
:103B4000E20005C019BC10922E021092230280914F
:103B5000E10080FF1AC08091E20080FF16C08091D2
:103B6000E2008E7F8093E2008091E200806180938A
:103B7000E2008091D80080628093D80019BC85E073
:103B800080932E0283E0809318018091E10084FFEE
:103B900037C08091E20084FF33C080E189BD82E1BB
:103BA00089BD09B400FEFDCF8091D8008F7D809340
:103BB000D8008091E1008F7E8093E1008091E20047
:103BC0008F7E8093E2008091E20081608093E2002A
:103BD00080912F02882311F084E007C08091E300D8
:103BE00087FD02C081E001C083E080932E028091B6
:103BF0002E02843011F081E001C082E08093180130
:103C00008091E10083FF2CC08091E20083FF28C0F7
:103C10008091E100877F8093E10082E080932E0213
:103C200010922F028091E1008E7F8093E1008091BD
:103C3000E2008E7F8093E2008091E20080618093B9
:103C4000E20042E060E080E00E94CA1E8091F00045
:103C500088608093F00081E08093180180931701C1
:103C6000FF91EF91BF91AF919F918F917F916F9154
:103C70005F914F913F912F910F900FBE0F901F902A
:103C800018952091E4003091E50095E64091EC0014
:103C9000842F817040FF23C08091E80080FD1DC00B
:103CA00080912E02882399F0853099F08091EB0065
:103CB00085FD11C04091E4005091E50024173507BF
:103CC00029F3915011F09A01E1CF84E0089582E048
:103CD000089583E0089581E0089580E0089540917B
:103CE000E80042FFDDCF0895089580911601089500
:103CF000FC01EE0FFF1F8E0F9F1FFC01E35AF94FCF
:103D00006183408322830895539A08958BB1877FFE
:103D10009BB198602FB7F894EDE5F6E036E0E93610
:103D2000F30789F0319148E09BB9000000C037FFEC
:103D30008BB9330F000000C000C000C08BB900C0B9
:103D40004A9591F7EBCF2FBF8FE594E00197F1F7FC
:103D500000C0000008958091300287FF11C080915B
:103D6000E80082FD05C080912E028111F8CF11C0BC
:103D70008091E8008B770BC080912E02882349F058
:103D80008091E80080FFF8CF8091E8008E778093E3
:103D9000E8000895982F973068F59093E9009817F8
:103DA00039F07091EC002091ED005091F00003C0CB
:103DB000242F762F50E021FD02C09F5FECCF309181
:103DC000EB003E7F3093EB003091ED003D7F309370
:103DD000ED003091EB0031603093EB007093EC001C
:103DE0002093ED005093F0002091EE0027FDE5CFE9
:103DF00080E008958F708093E90081E0089520911C
:103E00003602309137022617370748F061157105E1
:103E100039F42091E8002E772093E80001C0B90121
:103E2000FC0120E06115710579F180912E02882353
:103E3000F1F18530F1F18091E80083FD3CC0809183
:103E4000E80082FD2EC08091E80080FFEBCF20913A
:103E5000F3008091F20090E0922B6115710551F012
:103E60008830910538F421912093F1006150710957
:103E70000196F3CF21E0089709F020E08091E80057
